S105001E0001DB
S1048000007B
S123C000C735C717C73EC772C71DC725C72DC780C798C790C7A0C7F2C7E8C7DCC7E1C7FB67
S123C020C813C861C823C833C843C8E9C909C915C929C73BCA0CC93FC954C949CA68CA7435
S123C040CA7FC971C95DC97BC985C995C9D6CA02CA11CA2DCA3CCA4BC9E2C9F2C9C7C9AD7F
S123C060CA94CA98CA9ECAAFCAC2CAB5CAF8CACACB08CB6BCB80CB8ECBA0CB43CB4DCB268B
S123C080CB56D728D6D4D6FED716D73BD74ED760D76BD783D7A8D7B8D759D7D3D7E7D7F298
S123C0A0D7C8D7FDD808D813D825D833D841D6E3D869D88ED879D84FDCBADD98DD9CDDE103
S111C0C0DA3CCB59CB62DA15DA4BDA5C0000BD
S123C5000101010101CC0000FDFF028EFEFF7F003C8D1A20037EC6C0B680004A26F7CC804B
S123C52001CEC300ED008600A7097EC6C0CE002A4FA700088C003926F8CE10001C260886B7
S123C5403EA7097F00227F0023CC07C0DD261C39801D282086B0A72B860CA72D860597390D
S123C560BDDB30CC0000DD0CDD12DD148608970BCCC110DD16DD18DD1A8620B7C6A6CEC354
S123C58000C6208640A7098FC300108F5A26F6CEC300DF08CCC200ED00CCFE00ED04C30063
S123C5A001ED02830100ED06860AA7088620A709EF0CEF0EDC0CC30001DD0CED0ABDDA5C04
S123C5C0CEC5E7A6002706BDDB020820F6CE10001C200118CE3000180926FC1D20011D0083
S123C5E008CC0000DD2639496E74657261637469766520432020205620322E383220313124
S123C6002F372F39340A008D6B8D74816125F881732604863E2068368D513C18388D4C32FD
S123C6208172270D8177270F816327118162271B39A6008D4A2010188FE700200A188FA477
S123C64000A700EA00E700863E2034188F373C32331B331B97015D270C8D19A7009B0197B6
S123C66001085A26F496018D1620DC8D07368D0416328F39B6102E842027F9B6102F39F6BC
S123C680102EC48027F9B7102F39DE08A608970A1AEE00EE0218E600F7C69F1808FCC00062
S123C6A0FDC6A4BDFFFF20ED8620B7C6A6DC088FED021AEF00A60981402604EE0CDF08395F
S123C6C0963C260CCE10001F2E2005BDC60720F0120B02ECDE08EE0EDF088CC3002607DC3C
S123C6E01EC30001DD1EA609810026D4BDC68A810027CD814027C981202704860220028600
S123C700048D0220BB9701940B910126013996019A0B970B7EC67FEC02A300201CEC02A47E
S123C72000E4012014EC02AA00EA01200CEC02A800E8012004EC00E302ED020808398D26CE
S123C740A601E6033DDD00A600E6033DDB00D700EC013DDB00D7007D000727064F5F9300DF
S123C76020D7DC0020D37F00078D6308088D5F090939BDC766EC023CEE0002DF003820D720
S123C780EC00A3022705CC000020AECC000120A9EC02A3002EF520EEEC02A3002DED20E635
S123C7A03CEC002B1C26043808083937368605B7C7B5EC02380027030926FA380808ED0082
S123C7C0394F5FA30037368604B7C7B520E46D002A094F5FA300ED00730007396300630145
S123C7E0394F5FA300ED0039EC002705CC0001ED0039EC0027F64F5FED0039EC02E306DDE9
S123C80000E601E905A600A904ED04DC00ED06C6043A39EC06A302DD00E605E201A604A261
S123C8200020E6EC06A302E605E201A604A2002D1E2025EC02A306E601E205A600A2042DCF
S123C8400E2015EC06A302260FEC04A3002609C6063ACC0001ED0039C6063ACC0000ED004B
S123C860397F0007BDC8FF3CC6043ABDC8FFCE0000DF0038A603E6073DDD02A603E6063D44
S123C880D301DD01960089009700A602E6073DD301DD01960089009700A603E6053DD3004E
S123C8A0DD00A602E6063DD300DD00A601E6073DD300DD00EC033DDB00D700A602E6053DE7
S123C8C0DB00D700A601E6063DDB00D700A600E6073DDB00D700C6043ADC02ED02DC00ED04
S123C8E0007D000727028D0139CC0000A302DD00C600E2018600A200ED00DC00ED02396D43
S123C900002A058DE47300073918EC00180818080909ED003918EC020909ED0018EC001823
S123C9200818081808180820E718E600183A18A60009A70018095A26F518E600183A393C6B
S123C940CDEE00E600384F20C38FCDEE00EE028F0909ED008FCDEE00EE008F20AF18E6006C
S123C9603C3AEC00DD00EC02380909ED00DC00209D18E6003C3AEC003820933CA601CDEECD
S123C98000A70020083CEC00CDEE00ED0018083818080808393CEC00DD00EC02CDEE00ED98
S123C9A002DC00ED0038C6043A57183A39EC00DD00EC02D70718E6003C3AD607ED02DC00D9
S123C9C0ED0038080820C9EC00D70118E6003C3AD601ED0020B9A6013CEE02273FA7003848
S123C9E0202AA601B7C9EE3CEE0227301C00FF38201AA601B7C9FE3CEE0227201D00FF38D8
S123CA00200AEC003CEE022713ED00380808080839EC00DD00EC023CEE0426063886057EC6
S123CA20DDEDED02DC00ED0038080820DFEC003CEE0227E8E70038ED02080839EC003CEE95
S123CA400227D9ED0038ED02080839EC00DD00EC023CEE0427C6ED02DC00ED0038EC02EDD6
S123CA6004DC00ED020808393CEE0027AFE6004F38ED00393CEE0027A3EC0038ED00393C8D
S123CA80EE002798EC00DD00EC02380909ED02DC00ED003918EE00391AEE00080839EC0077
S123CAA0260618EE0008083918081808080839EC0026EF20F3EC0027EFCC0001ED0018EE98
S123CAC00039EC0026E218EE0039EC00DD0018EC00DF04D3048F1AEE002705DC00ED00399A
S123CAE0DE088640A7098621B7C6A6EC0C1AEE0E8FCDEF0C1AEF0E3918EC00DF00D3008F12
S123CB001AEE0027DB080839EC00DD00EC02DD0218EC00DF04D3048F1AEE0227C3DC00ED1E
S123CB2000DC02ED0239DF00DE08DC00A306CDA300250718081808DE00391809DE00860425
S123CB407EDDED8F18E3008F18081808393C323318E3007EC90CEE0039EC00DD3A080818B6
S123CB600839DC3A0909ED00180839EC003CEE021AA300382427E302C30002ED02080839C8
S123CB80EC003CEE021AA3003824120520E8EC003CEE021AA300382404050520D97EDDE7C7
S123CBA0EC003CEE021AA3003824F218A60018083D20C33CBDD644CE00003CDF3DDF3F7F7A
S123CBC000411830CDEE06A600BDCD0B2528812D260B73004108A600BDCD0B2519812E2696
S123CBE00B08A600BDCD0B24037ECC793131BDD64E38860F0D39A600BDCD0B2477BDCC8ABA
S123CC000824F37C003DA60008BDCD0B25F5812E260AA600BDCD0B24030820F68145270788
S123CC20816527037ECCCD08A600BDCD0B2515812D2706812B270520B318630008A600BDE0
S123CC40CD0B24A8803018A70108A600BDCD0B241418E601585818EB015880301B18A701AB
S123CC60088126228718A601186D002A01409B3D973D2059812E26A408A600BDCD0B249C08
S123CC808D0808258D7A003D20EF963E9743DC3FDD440579003E252C0579003E2526D34466
S123CCA036963E9943973E32251A0579003EDD3F2512E600C0304FD33FDD3F963E89002560
S123CCC003973E39DC44DD3F9643973E39CDEF06CE003DBDCD36272C963D18A701869697F6
S123CCE03DBDCD17186D01271B2A0BCECD41BDD6771860012006CECD45BDD677BDCD5518EF
S123CD006A0126F83131BDD64E383981302506813922020D390C39CE003D8D1A27147D0023
S123CD203E2B0FDC3F7A003D270A0579003E2AF5DD3F0C390D393736EC002602EC0232331E
S123CD40393DCCCCCD41200000BDCFF1BDD644BDCEC0BDD64E7D003D27057D0042260ACC72
S123CD6000009741DD3DDD3F39964198469741963D9B422A0924168606CEFFFF2009250D0B
S123CD808607CE0000DF40DF3DDF3F0D398B82973DCE00003C3C30BDCDCE6D002B0B6903D7
S123CDA06902690169007A003D6D032A13A6024CA702260CC601E3002404467C003DED0040
S123CDC038DF3E329740317D003D27B45F399645D6403DA7019644D6403DE300ED009645E5
S123CDE0D63F3DE300A70324026C026F006F019643D6403DE302ED029644D63F3DE302EDDF
S123CE000224026C019645D63E3DE302ED0224026C019643D63F3DE301ED0124026C0096C1
S123CE2044D63E3DE301ED0124026C009643D63E3DE300ED0039BDD644CED370BDD6777D53
S123CE4000412703730046BDCEF2BDD64E4FD63DC17F24035F201B53C3FF902F178FDC3E55
S123CE602001040926FC7D00412A074353C300012A020C3986090D39CC0000DD004FD63DC4
S123CE80C17F24035F203353C3FFA02F2F8F96405FDD00DC3E200704760000760001092660
S123CEA0F67D00412A147300007300014353DE0008DF002605C300012A020C3986090D3905
S123CEC0BDD2D8CE0045964280972A1BC6038B082A096F00095A26F66F0039C6804A2B03BD
S123CEE05720FAE400E7008D028D07964688FF974639963D260EDC42DD3DDC44DD3F9646FF
S123CF0097415F397D004227F9D641D84690422510811822ED183C36CE004318CE003E20FB
S123CF201740811822D0183C369642973D96469741CE003E18CE004317363636A80036173E
S123CF40A8013617A8023630A606E7061684074CC4185454543AE6034A27095666026601A7
S123CF60660020F45618A602A900974018A601A901973F18A600A902973E30A6062B1524E0
S123CF805A76003E76003F7600407C003D264CCCCD772053251B73004170004024087C001A
S123CFA03F26037C003E70003F24037C003E70003E7D003E2B252613963D80082326973D51
S123CFC0DC3F27207F0040DD3E20E67A003D271478004079003F79003E2AF01AEE07C609FA
S123CFE03A355F39CCCD801AEE07ED07C6073A35399646984197417D0042260586087ECD45
S123D000797D003D26055F7F004139963D904224052B057ECD802B1F8B7E973DDC3E934376
S123D0202B182606964090452B10DC3E04760040DD3E7C003D26037ECD77DC3EDE4308269B
S123D040010903183C18DE3EDF3E3CCE00003C3C309645D63F3DA703BDCDF818DF3EDC3FBF
S123D060A301DE4303DF3F7F003E383832331838D33EDD3E5F393CCE003DBDCD36260738B4
S123D080CC3000ED0039DE3D3CDE3F3C964136BDD644CE00003C3C3C1830CDEE0F86207D1F
S123D0A0004127057F0041862DA70008CDEF00CED1E0BDD677BDD1E42E19CED1DCBDD6775A
S123D0C0BDD1E42E16186A02CECD45BDD677BDCD5520DC186C02CECD4120F0CED370BDD637
S123D0E077BDCEF2D63DC07F50CB17200A74003E76003F7600405A26F4860118A70318A6F2
S123D100028B082B0A810824064A18A7038602800218A702186D032E15862ECDEE00A700D6
S123D12008186D0327058630A70008CDEF00CED1C7860718A705186F04DC3FA301DD3F965B
S123D1403EA200973E2505186C0420EDDC3FE301DD3F963EA900973E18A6048B303CCDEE76
S123D16000A70008186A032605862EA70008CDEF0038080808186A0526BCCDEE0009A6000A
S123D180813027F90818E602272A8645A70008862BA7005D2A0550862DA70008CDEF004F46
S123D1A0CE000A02378FCB30CDEE00E7000833CB30E700086F00383838BDD64E32974138CF
S123D1C0DF3F38DF3D38390F42400186A00027100003E800006400000A000001497423FE41
S123D1E04B18967F96462A12D6412A0EDC421A933D2617DC441A933F20109141260CDC3DAE
S123D2001A93422605DC3F1A93440784F424028A080639CE008EC3000026057ECD8009054B
S123D2202AFCDD3E7F00408F9741D73D5F394D2AE24353C30001CEFF8E20DBCE009EC3009F
S123D24000261118DE0026037ECD800978000179000059492AF5DD3E960097408F9741D727
S123D2603D5F394D2AD57300007300014353DE0008DF002603C30001CEFF9E20C1CE003D03
S123D280BDCD362601397D00412A04860A0D39BDD644860436DE3F3CDE3D3C18308D3996BD
S123D2A042807E4C2A03442003448B7E9742BDCFF1BDCEF27A003D8D1F18EC00DD3D18ECA5
S123D2C002DD3F186A0426E6DC42DD3DDC44DD3F383831BDD64E5F39DC3DDD42DC3FDD4498
S123D2E09641974639BDD644CED43FBDD677BDCFF1BDD64EDC3D1A8385B32B0B7D00412615
S123D300037ECD777ECD80BDD6449641367F0041BDCEC0DC4227068086544C26FC5C37CE16
S123D320D354BDD604CED350BDD6772003BDCD55306A0026F832324D2A0CBDD2D8CED598ED
S123D340BDD65EBDCFF1BDD64E5F39BDD64420EA402DF8543638EF1D37D00D0139500D0122
S123D3603AB60B613C0888893D2AAAAB3E2AAAAB3F0000003F8000003F800000FFBDD3999A
S123D380BDCD557ED2F48D11BDD644CED43FBDD677BDCD55BDD64E5F3996412704860C0D0D
S123D3A039963D27F8BDD6443C3C30BDD68F4FD63DC07F2A0143BDD22ECED43BBDD677BD2D
S123D3C0CD5530BDD677BDD68F867F97423C3C30BDD69DCED598BDD65EBDCEF230BDD67732
S123D3E0BDD68FCED437BDD65EBDCEF230BDD677BDCFF130BDD68FBDD2D8BDCD55CED41AB5
S123D400BDD60430BDD677BDCD55383830BDD677BDCEF23838BDD64E5F393E1D89D93E3A13
S123D4202E8C3E638E393E9249253ECCCCCD3F2AAAAB40000000FFBF8000003F3172183E71
S123D440DE5BD9860E0D39860D0D39BDD6449641367F0041CED598BDD677BDD1E42F07BDB5
S123D460D34B86FF20014F363C3C30BDD68FBDD2D8BDCD55CED4A2BDD60430BDD677BDCDB0
S123D480553838324D270CCED49EBDD677730041BDCEF2BDD5EE329741BDD64E5F393FC98B
S123D4A00FDBBCE2DD1B3D70F0F1BD8888893D9D89D9BDBA2E8C3DE38E39BE1249253E4CE8
S123D4C0CCCDBEAAAAAB3F800000FFBDD6444F2005BDD64486F036CED5B6BDD6772003BD23
S123D4E0CEF2964126F92003BDCEE7BDD1E42EF88D61240930A6002B04880FA7008D5424E2
S123D5000930A6002A04880FA7008D47240730A60088F0A700CED5FCBDD677BDCD55BDD2B1
S123D520D8BDCD553C3C30BDD69DA6042A05CED59D2003CED588BDD60430A604472403739F
S123D54000414D2B06BDD677BDCD55383831BDD64E5F397A0042BDD1E42E020C397C0042A4
S123D560730041BDCEF27A00420D39BDCEC0DC3DDE42DD42DF3DDC3FDE44DD44DF3F964162
S123D580D6469746D7415F393638EF1DB9500D013C088889BE2AAAAB3F800000FF37D00DE9
S123D5A001BAB60B613D2AAAABBF0000003F800000FF40490FDB43B40000BDD644BDD2D8A9
S123D5C0BDD4D1BDD56EBDD4CBBDCFF12407BDD64E860B0D39BDD64E5F397FFFFFFFBDD6A1
S123D5E044CED5FCBDD677BDCD55BDD64E39BDD644CED60020EECED5B27ED65E3C8EFA31BC
S123D60042652EE18FDE3D3CDE3F3C8F9641363CCC0000DD3DDD3FDD40201030A602974635
S123D620EC03DD44EC05DD42BDCD5530EE00BDD677BDCEF238C6043A3CA6004326DD30C6E8
S123D640073A3539383C3C8F3037367ED69D300808BDD67738313131316E00CED5987F00DC
S123D66041EC02DD3FEC00052403730041973D27020D56D73E5F397F0046EC02DD44EC00C2
S123D680052403730046974227020D56D74339DC3FED02DC3D58D1414656ED0039DC44ED8D
S123D6A002DC4258D1464656ED00397F00415F397D003E2705CC7F80DD3D4F5FDD3F397D71
S123D6C0003E27037300415F39BDD67708080808BDD65E393C183CEC00BDD22E1838380974
S123D6E00920AC3C183C0808BDD65E0909EE00BDD076183838EC00ED0408080808393C18AB
S123D7003CBDD65EBDCE7818383824037EDDEDED00DC00ED02393C183CEC02DD00EC00BDE9
S123D720D2631838387ED68F3C183CBDD65EBDCE4D18383824037EDDED205D3C183CBDD655
S123D740C9BDCEF2183838080808087ED68F3C183CBDD6C9BDCEE720EBA6008880A70039FD
S123D7603C183CBDD6C9BDCD5520093C183CBDD6C9BDCFF118383824037EDDED0808080831
S123D7807ED68F3C183CBDD6C9BDD1E4183838260CCC0001080808080808ED00390808084F
S123D7A00808086F006F01393C183CBDD6C9BDD1E41838382BDB20E53C183CBDD6C9BDD1CA
S123D7C0E41838382ECB20D53C183CBDD6C9BDD37D20A13C183CBDD65EBDD27D18383824F8
S123D7E0037EDDED7ED68F3C183CBDD65EBDD2F420EA3C183CBDD65EBDD2E520DF3C183C65
S123D800BDD65EBDD39920D43C183CBDD65EBDD38620C93C183CBDD65EBDD44B0736BDD54A
S123D820DE320620B73C183CBDD65EBDD5EEBDD4CB20A93C183CBDD65EBDD5EEBDD4D1204E
S123D8409B3C183CBDD65EBDD5EEBDD5BA208D8602E6019D47080839BDDB4FA600BDDC4627
S123D860A601BDDC4608082003BDDB4FA600BDDC46A601BDDC46080839BDDB4F3CEE008619
S123D88002E60027059D470820F738080839183CDF00BDDAA81A830051240C8621B7C6A692
S123D8A0DE001838180939DE00DC00C30002E300DD02830002DD04DE02EE000808A600268B
S123D8C0037EDA03812527037ED9F108A6008166261BDF02DE0409093CBDD65E380909DFCD
S123D8E004CEC100BDD076CEC1007ED9E38164267DDF0218CEC100DE040909DF04EC022AC6
S123D9000C862D18A7001808CC0000A302CE000A02378FCE000A02378FCE000A02378FCE46
S123D920000A02378FCE000A0237183C388601335D27064FCB30E70008334D27045D2706C2
S123D9404FCB30E70008334D27045D27064FCB30E70008334D27045D27064FCB30E70008AE
S123D96033CB30E700085FE700CEC10020758178262ADF02DE040909DF04A602BDDC2CBDF1
S123D980DAF0257217BDDAF0256CA603BDDC2CBDDAF0256217BDDAF0255C206181632611BC
S123D9A0DF02DE040909DF04A603BDDAF02547204C8162261EDF02DE040909DF04E60318C3
S123D9C0CE00085886308900BDDAF02529180926F2202A8173261ADF02DE040909DF04EEA4
S123D9E0020808A6002708BDDAF0250A0820F4200CBDDAF02409860ABDDB022006DE020852
S123DA007ED8BDDE00DC00C30002E3008FCC0000ED001838393CDC14C300011A931426FBEA
S123DA20C30001CE0000081A931426FA8F380909ED00CC000C0909ED007EC73E0909090923
S123DA400FDC14ED02DC120EED0039EC0008083C183CEE00AD00183838ED00390F3C183C3E
S123DA60B6103C84402605CEFF002003CEBF003CC6C03A18CEE0A71AEF0008083C32324DC5
S123DA8026F538CCC500EDFECCDE67EDE2CCDE5AEDE0CE10006F226F248600A7211C23185B
S123DAA01C22181838380E39960B84082707CC00F0DD062016DC1893162307830001DD06DF
S123DAC02009CC00F09316D318DD06960B84102705CC00F02012DC1A93162305830001202C
S123DAE007CC00F09316D31A1A93062302DC06393736BDDAA81A83000224040D3233393286
S123DB002001370F3CDE16088CC2002603CEC110DF16A700960B840827119C18260DDE186E
S123DB20088CC2002603CEC110DF1838330C0E39BDDBC9CC00389D478D2FC60C9D478D299D
S123DB408D308D258601970F8608971C4F971DCC00019D478D13C6069D478D0DC68F9D470D
S123DB608D073918CE011E200418CE0B29180926FC39CC00409D478602CEDB89E6009D47A1
S123DB808DE1088CDBC926F439000A1F1F0E04000000001111110F010E00000000000C04CD
S123DBA00800000F11110F010E00000C0C000C0C0000000C0C000C0408020006020202128A
S123DBC00C00000A0E04000000CEDBDE18CE0047A60018A7000818088CDC2C26F339FF00F3
S123DBE092CE10000F1D3C201D0010B700946F078104260F8601B710041C0010A6031D003D
S123DC0010201E8601B710041C0010A6031D001086FFA707B60094A704E7031C00101D0003
S123DC20101C3C20FE00920E3900000036840F8B30813A2B028B071632444444448B3081EF
S123DC403A2B028B0739BDDC2C371686029D47339D4739CE000A02378FCE000A02378FCEB2
S123DC60000A02378FCE000A02378FCE000A02379D47CC00019D47CC00079D47CC008F9DD9
S123DC8047860233CB309D4733CB309D47C62E9D4733CB309D4733CB309D4733CB309D477F
S123DCA0C66D9D47C6739D4739CC00029D478602E60027059D470820F739183CDF00CC7FED
S123DCC0FFDD04CEC3001AEE0E188CC3002607CCE400DD06200518EC04DD06EC0693063CBB
S123DCE0DE00A300382B091A93042E04DF02DD04188CC3002705183C3820CBDC041A837F88
S123DD00FF260486012015CEC310A609814027158FC300108F8C620026F08602DE00183822
S123DD2018097EDDED3C1838DE02EE0E1AEF0CCDEF0EDE021AEF0ECDEF0CEC0683000118E2
S123DD40ED04C30001DE00A30018ED06A60318A708EC0418ED00860018A709DC0CC300011F
S123DD60DD0C18ED0ADC00E306C30008EE068F09DF0018DF0218EE0436A60018A7003209D3
S123DD80180983000126F1DE0218081AEF02DE0009DC0CED00183839862020513CEC00DD57
S123DDA000CEC300EC0A1A9300270EEE0E8CC30026F238CC0001ED00399C082604387ECA1A
S123DDC0E0183C8640A7098621B7C6A6EC0C1AEE0E8FCDEF0C1AEF0E183838CC0000ED000E
S123DDE0398621B7C6A6391809860320003CDE084D2602861FA70997018621B7C6A6960134
S123DE0081202431CEDE37A6002708BDDAF025F70820F44FD601C00A25034C20F9CB0A8BB4
S123DE2030BDDAF025FB178B30BDDAF025FB860ABDDAF025FB38390A52554E54494D452098
S123DE404552522000CE1000DC28E316ED161D237FB610008880B710003BCE1000DC26E385
S123DE601EED1E1D23F73BCE1000CC07D0E31CED1C1D23EFA62236A7220EDE1408DF142663
S123DE8005DE1208DF127A000A26058621B7C6A686049D47848027037EDF729615843F2618
S123DEA040960F8101223A0F4FC6CF9D47DC1E1A8300642D0BCC0000DD1E961C880C971CD1
S123DEC0961C84082704C6002002C60786029D474FD611C1102502CB30CA809D470E7EDFF2
S123DEE0729639840126037EDF72960F8102245EDE1A9C16277C088CC2002603CEC110DF6C
S123DF001AE600960F81002634C10A26068601970F205F9611811F27594C97118111260760
S123DF204F37C6C09D4733C120250CC17F2208CEDFB4C0203AE60086029D47203581012674
S123DF400DD710FCDFA29D478602970F2024810A2712CEDFA2D60F3AEC009D47960F8B02C2
S123DF60970F200E8600970F86019711D610C10A26B5963984042725CE1000962248240736
S123DF801C00108B0120031D0010972296234824071C00208B0120031D0020972332B710B5
S123DFA0223B0001000600CF020000020011495557777FFF202122232425262728292A2B69
S123DFC0022D2E2F3031323334353637383904053C3D3E3F404142434445464748494A4B63
S123DFE04C4D4E4F505152535455565758595A5B5C5D5E5F60616263646566036869066B75
S123E0006C6D6E6FF0F172737475767778017A7B7C7D7E7F18CE03E8180926FCCE10001F35
S123E020000433CC1BE61F00042C83000126F7203937368D56CC00029D47CEE05F8602E612
S123E0400027059D470820F732BDDC4632BDDC468602C6299D47CE10001C28204F06CF2A80
S123E06048616C7465642A2028008D1FCEE07BBDDCA9CE10001D23FB8D163B2D504F574562
S123E0805220474C495443482D20008601979039860E979039CE80004F5FE3008FC30002F4
S10BE0A08F8CFF0226F4393BCA
S123BFC0E0A7E0A7E0A7E0A7E0A7E0A7E0A7E0A7E0A7E0A7E0A7E0A7E0A7E0A7E0A7E0A7ED
S123BFE0DE5ADE67E0A7E0A7E0A7E0A7E0A7E014E0A7E0A7E0A7E0A7E0A7E0A7E0A7C500B3
S123FFC0E0A7E0A7E0A7E0A7E0A7E0A7E0A7E0A7E0A7E0A7E0A7E0A7E0A7E0A7E0A7E0A7AD
S123FFE0DE5ADE67E0A7E0A7E0A7E0A7E0A7E014E0A7E0A7E0A7E0A7E0A7E0A7E0A7C50073
S105FF020000F9
S105FF000252A7
S9030000FC
